:060000002500A304A50B7E
:10034A00D10C02003B0C0600A4047D0066000602E4
:10035A003B0E3D00F20BC50C210001024307B20B14
:10036A00040CA6010000B00BC60C210001024307D1
:10037A00BB0B040CA6010000B90BC40C210001023E
:10038A004307C40B040CA6010000C20BD60C0200E2
:10039A00DC0C3F00000C6606010C3E001F02210027
:1003AA0001024307D50B040CA601000C6606010CDA
:1003BA00270068009E0108014306D30BBF021F02F3
:1003CA00FD0F4307CF0BCD0BC70C210001024307DA
:1003DA00EB0B040CA6010000E90B1D02300F4306CB
:1003EA00CB0B080F4306B00B020F4306B90B010FE4
:0603FA004306C20BE90BF3
:021FFE000A00D7
:00000001FF
